:103800000C942A1C0C94451C0C94451C0C94451CCF
:103810000C94451C0C94451C0C94451C0C94451CA4
:103820000C94451C0C94451C0C94451C0C94451C94
:103830000C94451C0C94451C0C94451C0C94451C84
:103840000C94451C0C94451C0C94451C0C94451C74
:103850000C94451C11241FBECFE5D4E0DEBFCDBFC4
:1038600010E0A0E6B0E0EAE5FFE302C005900D92AB
:10387000A036B107D9F711E0A0E6B0E001C01D9273
:10388000A43AB107E1F70C94721F0C94001C0F933B
:10389000EF93FF933ED0FC01062F35D0FF91EF91BF
:1038A0000F9108950F930F921F92EF93FF9331D0D2
:1038B000FC010B0101E027D0FF91EF911F900F90C9
:1038C0000F9108950F930F92EF93FF9322D0FC0175
:1038D00060FD67BFC895802DE395C895902DFF9139
:1038E000EF910F900F9108950F930F9212D0082E21
:1038F00009E009D00F900F9108950F930AD001E1CC
:1039000002D00F910895E199FECF07BFE895FFFF20
:10391000000007B700FDFDCF089587E089B9549AEC
:10392000539A08958CB19927089540E050E04817C4
:10393000590750F422E537E000002150304037FFAE
:10394000FBCF4F5F5F4FF3CF08958BB199278078FE
:10395000907008955498539808950E94AA1C0C944E
:10396000000008958CB95E9BFECF5E9A08950E9478
:10397000A51C8823E1F30E94921C803219F481E097
:1039800090E0089585E10E94B21C80E090E00895E7
:103990000895EF92FF920F931F93CF93DF937B01D4
:1039A000C0E0D0E0C617D70770F48C010E94A51CB8
:1039B0008823E1F30E94921CF80181938F012196E4
:1039C000CE15DF0598F381E090E0DF91CF911F9154
:1039D0000F91FF90EF90089590E0282F3327213822
:1039E000310589F02238310524F42038310549F0B9
:1039F0000DC02238310549F02839310539F493E0FA
:103A000005C092E003C091E001C092E1892F99279F
:103A1000089540E050E06091A0007091A100461729
:103A20005707E8F4E2EAF0E08091A2018EBB8091B2
:103A3000A2019091A301292F33272FBB01969093C8
:103A4000A3018093A20180818DBBE29AE19AE19962
:103A5000FECF4F5F5F4F31964617570728F3089503
:103A60000F931F93CF93DF9300E010E08091A000AD
:103A70009091A10008171907D8F4C2EAD0E080910C
:103A8000A2019091A301880F991F60E0800F911F00
:103A90000E94621C8883892F992789830E5F1F4F9C
:103AA00022968091A0009091A1000817190738F381
:103AB000DF91CF911F910F9108958091A000909177
:103AC000A1000097C1F0E2EAF0E0AC018091A20110
:103AD0008EBB8091A2019091A301292F33272FBB88
:103AE00001969093A3018093A201E09A8DB38193F4
:103AF0004150504059F708950F931F93CF93DF9390
:103B00008C016115710541F0EB01F80181918F0184
:103B10000E94B21C2197C9F781E090E0DF91CF911C
:103B20001F910F910895EF92FF920F931F93CF93E0
:103B3000DF93C0E0D0E08E017E01CFE7D0E0F092CD
:103B4000A301E092A20163E0C8010E94471C2197F3
:103B500080E490E0E80EF91E00581F4FD7FFEFCF2A
:103B60000E947D1CDF91CF911F910F91FF90EF90EC
:103B70000895EF92FF920F931F93CF93DF9300E08E
:103B800010E08091A0009091A1000817190708F09B
:103B900047C0EE24FF24E801CD55DF4FF801EE5574
:103BA000FF4FEE0DFF1D4081888122969927382F07
:103BB0002227240F311D8091A2019091A301880F2B
:103BC000991FB9018E0D9F1D0E94521C82E090E04A
:103BD000E80EF91E90E8E916F10400F38091A201C5
:103BE0009091A301880F991F63E0800F911F0E949D
:103BF000471C8091A2019091A301880F991F65E055
:103C0000800F911F0E94471C0E947D1C00581F4F6F
:103C10008091A0009091A1000817190708F4B9CF6E
:103C2000DF91CF911F910F91FF90EF900895CF9367
:103C3000C0E069E081E090E00E94621C84FF03C064
:103C40008F7E0E94741C0E94A51C8823E1F30E94B1
:103C5000921C992782359105DCF4803591050CF092
:103C600054C08134910509F45AC0823491053CF462
:103C70008033910509F449C0C19759F12FC18234AD
:103C8000910509F45FC08534910509F45EC026C131
:103C90008635910509F4EDC0873591054CF48235E0
:103CA000910509F461C08535910509F465C016C117
:103CB0008437910509F4A0C0853791052CF484362A
:103CC000910509F472C00AC18537910509F4C1C094
:103CD00005C10E94B71C882309F4B5CF84E10E9476
:103CE000B21C81E40E94B21C86E50E94B21C82E5EF
:103CF0000E94B21C80E20E94B21C83E50E94B21CAA
:103D000084E50E94B21C8BE406C00E94B71C882385
:103D100009F499CF84E10E94B21C80E1E0C061E027
:103D200070E080E690E00E94C91C0E94B71C8823C6
:103D300009F489CF84E10E94B21C809160000E9446
:103D4000EC1CE9CF64E170E00AC061E070E080E65D
:103D500090E00E94C91C809160009927BC0180E618
:103D600090E00E94C91CD1CF0E94B71C882309F49F
:103D70006ACF0E94931DCECF62E070E080E690E0B3
:103D80000E94C91C0E94B71C882309F45CCF2091B3
:103D90006000809161009927982F8827820F911DDC
:103DA0009093A3018093A201B5CF63E070E080E619
:103DB00090E00E94C91C20916100809160009927C9
:103DC000982F8827820F911D9093A1008093A000C7
:103DD000BC0182EA90E00E94C91C0E94B71C8823A3
:103DE00009F431CF80916200863419F40E94B91D24
:103DF00091CF0E94091D8ECF63E070E080E690E0D5
:103E00000E94C91C20916100809160009927982F21
:103E10008827820F911D9093A1008093A0000E949B
:103E2000B71C882309F40FCF80916200863419F4FF
:103E30000E94301D02C00E945D1D84E10E94B21CE0
:103E40006091A0007091A10082EA90E00E947C1D28
:103E500064CF0E94B71C882309F4F5CE84E10E9448
:103E6000B21C8EE10E94B21C84E90E94B21C83E065
:103E700052CF64E070E080E690E00E94C91C0E948E
:103E8000B71C882309F4DFCE84E10E94B21C809124
:103E90006000803531F480916100882361F4C82F7F
:103EA00017C0883531F480916100883061F4C3E037
:103EB0000FC0803531F480916100883049F4C2E050
:103EC00007C0883529F480916100882309F4C1E096
:103ED00069E08C2F99270E94621C1DCF85E10E940A
:103EE000B21CB1CECFE5D4E0DEBFCDBFCEE1F894B9
:103EF0008EEF91E00E94A41F843B59F48FEF91E074
:103F00000E94A41F833C29F48DEF91E00E94A41F1E
:103F100081BF0E948D1C0E94921C84E690E00E944A
:103F2000951C0E94A51C882321F4C150C8BBCC233A
:103F3000A1F7CC2319F00E94171E02C00E94AD1CED
:103F400080E090E00C94AC1FE199FECF9FBB8EBB4C
:0A3F5000E09A99278DB30895FFCF82
:0400000300003800C1
:00000001FF
